:0200000067296E
:08000800F2288207503469342C
:1000100063342034543465346D3470346534723450
:100020006134743475347234653420344C346F3434
:1000300067346734653472340D340A3428344334F9
:1000400029344D3461347234203432343034303415
:1000500030342C34203456344B3431345A34443414
:100060004A342E340D340A340D340A3444345334B3
:10007000313420342D34203430343D345234613422
:1000800077342C34203431343D344434653467348F
:1000900043340D340A3444345334323420342D3450
:1000A000203430343D3443346F346E347434693426
:1000B0006E346F34753473342C34203431343D3421
:1000C0004C346F34673420340D340A3444345334A0
:1000D000333420342D342034533461346D3470344F
:1000E0006C346534203452346134743465342034D3
:1000F00030340D340A3444345334343420342D3401
:100100002034533461346D3470346C3465342034AD
:100110005234613474346534203431340D340A344B
:100120000D340A34533461346D3470346C346534B6
:100130002034723461347434653473343A340D3499
:100140000A340D340A34313431343D3435345334C7
:1001500065346334283435342E343534203448340F
:100160007234733420344D346134783429340D348E
:100170000A34313430343D3431344D3469346E34E2
:10018000283432342E3438342034443461347934D1
:10019000733429340D340A34303431343D34353439
:1001A0004D3469346E34283431343434203444349A
:1001B00061347934733429340D340A3430343034B2
:1001C0003D34333430344D3469346E34283438346B
:1001D00035342034443461347934733429340D3463
:1001E0000A340034C3000308C40006088B01C501AB
:1001F000C6018610061807296430A123C50A4508E0
:10020000CE3E031DFA28FF30C6008614FA28461C8D
:100210001929C001BF01003089003F0888005D2214
:1002200001308900400888005D228610C501002841
:100230006029573052237230522369305223743070
:100240005223653052233D3052233F083423400867
:1002500034230D3052230A30522354305223453078
:1002600052234D305223503052235F3052234430BA
:1002700052234130522354305223413052230D3007
:1002800052230A3052233F08003E031948295F29B0
:100290004008003E031D5F294E3052234F30522349
:1002A00020305223443052234130522354305223C1
:1002B000413052230D3052230A3052236029C92283
:1002C0004408830090308B00C30E430E09008B015D
:1002D0008316FD308600003085003F308100831298
:1002E00000305722BF0001305722C0005222F822AE
:1002F000522290308B007C293F08E03E031D832969
:1003000090308B006300861AC1290608C039003E70
:10031000031D8B2996230608C039803E031D9129B1
:1003200086230608C039C03E031D97297623060898
:10033000C039403E031D9D296E232222CC30292244
:1003400044302922FA30A123F030A1235222222264
:10035000CC302922BE3029228B013522B700B822A9
:100360003522B800B822003089003F0888005D229D
:1003700001308900400888005D2290308B002222E5
:100380007C292222CC30292244302922FA30A12390
:10039000F030A12352222222CC302922BE30292241
:1003A000061ADD293522B7003522B80006230D30A4
:1003B00052230A30522322227C293522B7003522CB
:1003C000B8003522B9003522BA003522352235224F
:1003D000BB003522BC00222244305223613052231C
:1003E00074305223613052233A3052233808342378
:1003F0002C305223370834232C305223390834232D
:100400002C3052233A0834232C3052233B08342317
:100410002C3052233C0834230D3052230A3052230F
:100420007C29831605148312080005108316051015
:100430008312080015221E2A152211221430AB2324
:100440001122080015229630AB2311226430AB2311
:100450000800B4000830B600B40C0318312A1A2280
:10046000322A1C22B60B2C2A08000830B6001522AE
:100470001122000000000000000000000000000049
:10048000000000000000000000000000000000006C
:100490000314051C0310B40C1430AB23B60B372A1D
:1004A0003408080086140A30A12386100800890049
:1004B000831608148312080808008316880108159B
:1004C00055308900AA30890088148818652A0815D3
:1004D000081283120800051508000511080083168C
:1004E0008515831208008511831685118312080073
:1004F0006B22AB23AB236D22AB23AB2308006D2211
:100500006F226B2273226D22AB2308006D227322AF
:100510006B226F226D22AB2308006F227822080025
:10052000732278220800B4000830B6000310B40D1E
:1005300003189E2A732278226F22A02A6F22782223
:10054000B60B962A8D2208000830B6006F226B2267
:10055000AB23851DAD2A0314AE2A0310B40D6D2202
:100560000000000000000000B60BA72A34080800B5
:10057000BE007F22A03093223F089322400893229E
:100580003E08932286221430A123C00A0319BF0A11
:1005900008000D3052230A3052233F08C1004008A2
:1005A000C200C10A7F22A030932200309322003083
:1005B00093227F22A1309322A422B7009022A4226A
:1005C000B8000623C20BE72AC10BE72AEB2AC20BAD
:1005D000F22AC10BF22A8D2286220D3052230A30D4
:1005E0005223080090220D3052230A305223DC2A75
:1005F0000D3052230A3052230030B3003308052057
:10060000003E031908005223B30AFE2A03308A0071
:100610002D30381C2B3052233708381837097F39D2
:10062000B70037080139B900370C7F39B7003708F0
:100630009C3E031C1E2BB700313052233708B001FB
:10064000B00AF63E0318202B0A3EB003B70030086C
:10065000402352233708402352232E305223353073
:10066000391C303052230800BD0003308A003D0E93
:100670000F39402352233D080F39402352230800ED
:100680008207303431343234333434343534363410
:100690003734383439346134623463346434653423
:1006A00066345834B4000830B60085143130AB23BA
:1006B000B40C03185D2B85145F2B85100000B60B5E
:1006C000562B3430AB2385106830AB230800B000C4
:1006D000B100B10B692BB00B682B08001E30B000C5
:1006E0008623B00B702BC430A12308004730B10023
:1006F0009623B10B782B2C30B2006430A123B20BBF
:100700007D2B4D30A1230130AB2308000D30B1000B
:100710009623B10B882B1430B200FA30A123B20B10
:100720008D2BC930A1239630AB2308001030B200C6
:10073000FA30A123B20B982B9B30A1239830AB2326
:100740000800C700F930AB2300000000C70BA22B44
:100750000800F9300000FF3E00000000000000002B
:0A07600000000000031DAB2B080091
:02400E00F23F7F
:00000001FF
